:100000000AC022C021C020C01FC07CC05BC01CC071
:100010001BC01AC019C011241FBECFEDCDBF10E008
:10002000A0E6B0E0E0EAF7E003C0C89531960D9293
:10003000A639B107D1F710E0A6E9B0E001C01D92E2
:10004000A23AB107E1F7E9C1DBCF18BA8FEF87BB5E
:100050008CE782BB80E481BB089589E189B988E19E
:100060008AB908955D9BFECF8CB908958AE0FADFC6
:100070008DE0F8DF0895FF920F931F93CF93DF93E6
:10008000FF242F2DD92FC82F082F192F015F1F4FA5
:100090008991882339F0F82E822FE4DF2F2D0C1759
:1000A0001D07B4F78091A100882311F08EE2DADFFA
:1000B0008F2DD8DF1092A100DF91CF911F910F916A
:1000C000FF9008951F920F920FB60F9211248F93F5
:1000D0009F9380919A0090919B00409719F48FEF25
:1000E00080939C0080919A0090919B000196909340
:1000F0009B0080939A009F918F910F900FBE0F905D
:100100001F9018951F920F920FB60F9211242F93E4
:100110003F934F935F936F937F938F939F93AF938F
:10012000BF93EF93FF938091960090919700A091D9
:100130009800B091990020E030E040E85FE3682F3C
:10014000792F8A2F9B2FBAD1B92FA82F972F862FBF
:100150008093960090939700A0939800B093990095
:10016000FF91EF91BF91AF919F918F917F916F918F
:100170005F914F913F912F910F900FBE0F901F9065
:10018000189585E083BF86E08EBD82E889BF08951B
:1001900013BE1EBC0895EF92FF920F931F9360E071
:1001A00070E080E090E01DBC1CBC10929B0010929F
:1001B0009A0010929C0012BE609396007093970074
:1001C0008093980090939900DCDF789480919C0054
:1001D000882331F49CE592BB80919C008823D9F35D
:1001E000F894D6DF8CE182BB0CB51DB5802F912F22
:1001F000AA2797FDA095BA2F682F792F8A2F9B2FBA
:1002000002D217FF05C020E030E040E857E456D1A5
:10021000262F372F482F592F60E070E080E090E0C4
:100220004DD1E62EF72E082F192F80919600909130
:100230009700A0919800B091990020E030E040E84C
:1002400057E4682F792F8A2F9B2F35D2B92FA82FEB
:10025000972F862F282F392F4A2F5B2F912F802FF2
:100260007F2D6E2D2BD1B92FA82F972F862F20E011
:1002700030E04AE754E4682F792F8A2F9B2F1BD256
:10028000B92FA82F972F862F20E030E44BE854E4B5
:10029000682F792F8A2F9B2F53D11F910F91FF9099
:1002A000EF900895AF92BF92CF92DF92EF92FF92BC
:1002B0000F931F93CF93DF93CDB7DEB760970FB641
:1002C000F894DEBF0FBECDBF66DFA62EB72EC82EB8
:1002D000D92E20E030E04DE154E4EDD1B92FA82F24
:1002E000972F862F282F392F4A2F5B2F67EB73E428
:1002F0008AEB91E525D1B92FA82F972F862F282F8C
:10030000392F4A2F5B2F682F792F8A2F9B2FD3D11C
:10031000B92FA82F972F862F20E030E04AE754E42A
:10032000682F792F8A2F9B2F0BD1E62EF72E082FBF
:10033000192F84990EC060939D0070939E00809346
:100340009F009093A0001092A10090DE80E690E0C4
:1003500052C080919D0090919E00A0919F00B0910D
:10036000A000282F392F4A2F5B2F912F802F7F2D10
:100370006E2DA3D02BD161302AEC72072AE98207B7
:100380002BE3920720F072DE89E690E034C02AE089
:1003900030E04C2F5D2F4F5F5F4F57D067DE66DE3A
:1003A000839904C08FE690E066DE06C087E790E0A0
:1003B00062DE81E08093A1008C2F9D2F01965BDE91
:1003C00055DE8FE790E057DE9D2D8C2D7B2D6A2D1D
:1003D000FDD0B92FA82F972F862F2AE030E04C2F81
:1003E0005D2F4F5F5F4F682F792F8A2F9B2F2DD066
:1003F0008C2F9D2F01963FDE60960FB6F894DEBFDE
:100400000FBECDBFDF91CF911F910F91FF90EF9065
:10041000DF90CF90BF90AF900895CFEDD0E0DEBFDA
:10042000CDBF13DE1ADE80E090E0A0E0B0E0809364
:100430009D0090939E00A0939F00B093A000ABDE20
:1004400087E890E018DE2EDFFECFE42FF52FCF9364
:10045000FF93EF932230D4F02532C4F4C22F2C2F17
:10046000332744275527FF93EF9373D1EF91FF91E3
:10047000605D6A330CF0695D6193622F732F842F86
:10048000952F605070408040904049F710828F91C6
:100490009F91CF9100C0A82FB92FE82FF92F01907D
:1004A0000020E9F73297AE17BF0730F47C916081E6
:1004B000708331976D93F7CF08955058192ECDD092
:1004C00001D0B0C0BA176207730784079507B1F16E
:1004D00088F40EF410940B2EBA2FA02D062E622F46
:1004E000202D072E732F302D082E842F402D092EFE
:1004F000952F502DFF275523B9F0591B49F0573E32
:1005000098F0469537952795A795F0405395C9F7EC
:1005100076F0BA0F621F731F841F30F487957795AA
:100520006795B795F040939517FA0F2E0895BF1B66
:10053000BB27BA0B620B730B840BF6CFDEF6B9C088
:100540008CD001D06FC0552359F0992369F09F5783
:100550005F57951B33F442F4903811F4915805C05D
:1005600079C091589F3F09F4A4C0BB27112462179A
:100570007307840730F4660F771F881FBB1F9150E5
:1005800098F311D00F920FD00F920DD0A0E826173C
:10059000370748071B0609F0A048BA2F602D7F9146
:1005A0008F9100240895A0E8002462177307840740
:1005B000B10528F0621B730B840BB1090A2A660F80
:1005C000771F881FBB1FA69581F7089597FB51D011
:1005D0009F3738F0FEE9F91B982F872F762F6B2F66
:1005E00005C064C09695879577956795F150D0F7CB
:1005F0003EF490958095709561957F4F8F4F9F4FFA
:100600000895E89403C097FB0EF4F3DFB62F672F2D
:10061000782F892F9EE9002405C09A95BB0F661F8D
:10062000771F881F11249923A1F08823B2F79F3FD9
:1006300059F0BB0F48F421F4002011F460FF04C00E
:100640006F5F7F4F8F4F9F4F881F9795879597F9C3
:1006500008952CC09FEF80EC0895052E092607FA17
:10066000440F551F5F3F79F0AA27A51708F051E006
:100670004795880F991F9F3F31F0BB27B91708F0A6
:1006800091E0879508959F919F911124E3CF97FB67
:10069000880F991F9F3F31F0BB27B91708F091E0F1
:1006A000879508959F919F911124D4CF662777272E
:1006B000882799270895D1DF01D0B4CF992339F045
:1006C000552329F09F575F57950F13F4CAF1F1CFC7
:1006D00091589F3FE1F3A62F00241124BB276627E2
:1006E0005527F8E0A69520F4020E131EB41F651FCF
:1006F000220F331F441F551FFA95A1F7F8E0E72F8B
:100700007727F8E0E69520F4130EB41F651F7A1FD3
:10071000330F441F551FAA1FFA95A1F7F82F8827FA
:10072000F69520F4B40F651F7A1F8E1F440F551FD6
:10073000AA1FEE1FFF23A1F788231AF4939539F41B
:1007400089CF000C111CBB1F661F771F881F012853
:100750000895A1E21A2EAA1BBB1BEA2FFB2F0DC086
:10076000AA1FBB1FEE1FFF1FA217B307E407F50761
:1007700020F0A21BB30BE40BF50B661F771F881F3D
:10078000991F1A9469F76095709580959095262F1A
:10079000372F482F592F6A2F7B2F8E2F9F2F089589
:1007A0005A45524F205345540052414E474500434D
:1007B000287066293D20004C287548293D200046B8
:1007C00028487A293D20004C436D657465723037A6
:0607D00030323137410018
:00000001FF
